 flexcan

 Timestamp is 4fb04cc1 (Mon May 14 12:07:29 2012)

 Preferred load address is 10000000

 Start         Length     Name                   Class
 0001:00000000 00000004H .CRT$XCA                CODE
 0001:00000004 00000004H .CRT$XCZ                CODE
 0001:00000008 00000004H .CRT$XIA                CODE
 0001:0000000c 00000004H .CRT$XIZ                CODE
 0001:00000010 00000004H .CRT$XPA                CODE
 0001:00000014 00000004H .CRT$XPZ                CODE
 0001:00000018 00000004H .CRT$XTA                CODE
 0001:0000001c 00000004H .CRT$XTZ                CODE
 0001:00000020 000001e8H .rdata                  CODE
 0001:00000208 00000024H .rdata$debug            CODE
 0001:0000022c 0000261cH .text                   CODE
 0001:00002848 00000018H .xdata                  CODE
 0001:00002860 0000003cH .idata$2                CODE
 0001:0000289c 00000014H .idata$3                CODE
 0001:000028b0 000000d0H .idata$4                CODE
 0001:00002980 000000a6H .idata$6                CODE
 0001:00002a30 000000b5H .edata                  CODE
 0002:00000000 000000d0H .idata$5                DATA
 0002:000000d0 0000044cH .data                   DATA
 0002:00000520 00000014H .bss                    DATA
 0003:00000000 00000190H .pdata                  DATA

  Address         Publics by Value              Rva+Base       Lib:Object

 0000:00000000       ___safe_se_handler_count   00000000     <absolute>
 0000:00000000       ___safe_se_handler_table   00000000     <absolute>
 0001:00000000       __xc_a                     10001000     corelib0:crt0init.obj
 0001:00000004       __xc_z                     10001004     corelib0:crt0init.obj
 0001:00000008       __xi_a                     10001008     corelib0:crt0init.obj
 0001:0000000c       __xi_z                     1000100c     corelib0:crt0init.obj
 0001:00000010       __xp_a                     10001010     corelib0:crt0init.obj
 0001:00000014       __xp_z                     10001014     corelib0:crt0init.obj
 0001:00000018       __xt_a                     10001018     corelib0:crt0init.obj
 0001:0000001c       __xt_z                     1000101c     corelib0:crt0init.obj
 0001:0000003c       ??_7?$Buffer_t@VDuplicateTraits_t@detail@marshal@ce@@@detail@marshal@ce@@6B@ 1000103c     driver.obj
 0001:00000040       ?dwCANRegisterValues@FlexCAN@@0QBKB 10001040     flexcan.obj
 0001:00000088       ??_C@_1BA@MNOLBALH@?$AAB?$AAi?$AAt?$AAr?$AAa?$AAt?$AAe?$AA?$AA@ 10001088     settings.obj
 0001:00000098       ??_C@_1M@KEKDJCFI@?$AA?$CF?$AAs?$AA?$CF?$AAd?$AA?3?$AA?$AA@ 10001098     settings.obj
 0001:000000a4       ??_C@_1BI@BHLBGEOK@?$AAP?$AAr?$AAi?$AAo?$AAr?$AAi?$AAt?$AAy?$AA2?$AA5?$AA6?$AA?$AA@ 100010a4     settings.obj
 0001:000000bc       ??_C@_1O@GBAEOCCH@?$AAP?$AAr?$AAe?$AAf?$AAi?$AAx?$AA?$AA@ 100010bc     settings.obj
 0001:000000cc       ??_C@_1M@EENNDIOJ@?$AAI?$AAn?$AAd?$AAe?$AAx?$AA?$AA@ 100010cc     settings.obj
 0001:000000d8       ?canSetup@FlexCAN@@0QBUCAN_SETUP@@B 100010d8     flexcan_pdd:pdd.obj
 0001:0000022c       ?Unmarshal@MarshalledBuffer_t@@QAAJXZ 1000122c f i driver.obj
 0001:00000288       DllMain                    10001288 f   driver.obj
 0001:000002a0       ?Deinit@@YAHPAUDRIVER_INFO@@@Z 100012a0 f   driver.obj
 0001:000002f4       ?Open@@YAPAUOPEN_INFO@@PAUDRIVER_INFO@@KK@Z 100012f4 f   driver.obj
 0001:00000374       ?Close@@YAHPAUOPEN_INFO@@@Z 10001374 f   driver.obj
 0001:000003c8       ?Read@@YAKPAUOPEN_INFO@@PAEK@Z 100013c8 f   driver.obj
 0001:000003d0       ?Write@@YAKPAUOPEN_INFO@@PAEK@Z 100013d0 f   driver.obj
 0001:000003d8       ?Seek@@YAKPAUOPEN_INFO@@JK@Z 100013d8 f   driver.obj
 0001:0000043c       ?Free@?$Buffer_t@VDuplicateTraits_t@detail@marshal@ce@@@detail@marshal@ce@@QAAJXZ 1000143c f i driver.obj
 0001:00000484       ?Allocate@?$Buffer_t@VDuplicateTraits_t@detail@marshal@ce@@@detail@marshal@ce@@QAAJPAXKK@Z 10001484 f i driver.obj
 0001:000004cc       ?Marshal@MarshalledBuffer_t@@QAAJPAXKKHH@Z 100014cc f i driver.obj
 0001:00000560       ?Init@@YAPAUDRIVER_INFO@@PAX@Z 10001560 f   driver.obj
 0001:000005f8       ??_E?$Buffer_t@VDuplicateTraits_t@detail@marshal@ce@@@detail@marshal@ce@@UAAPAXI@Z 100015f8 f i driver.obj
 0001:000005f8       ??_G?$Buffer_t@VDuplicateTraits_t@detail@marshal@ce@@@detail@marshal@ce@@UAAPAXI@Z 100015f8 f i driver.obj
 0001:0000062c       ?IOControl@@YAHPAUOPEN_INFO@@KPAEK1KPAK@Z 1000162c f   driver.obj
 0001:0000096c       ?CleanInterruptHandler@FlexCAN@@AAAXXZ 1000196c f   flexcan.obj
 0001:00000a38       ?GetClockFreq@FlexCAN@@AAAKXZ 10001a38 f   flexcan.obj
 0001:00000a70       ?EnableMBInterrupt@FlexCAN@@AAAXEH@Z 10001a70 f   flexcan.obj
 0001:00000ae8       ?FindFreeMB@FlexCAN@@AAAEXZ 10001ae8 f   flexcan.obj
 0001:00000b34       ?ReadMessageBuffer@FlexCAN@@AAAHPAUCAN_PACKET@@@Z 10001b34 f   flexcan.obj
 0001:00000cc0       ?SetRxMask@FlexCAN@@AAAXEK@Z 10001cc0 f   flexcan.obj
 0001:00000d18       ?EnableDoze@FlexCAN@@QAAXH@Z 10001d18 f   flexcan.obj
 0001:00000d60       ?DozeEnabled@FlexCAN@@QAAHXZ 10001d60 f   flexcan.obj
 0001:00000d80       ?BlinkLED@FlexCAN@@AAAHW4CAN_LEDS@@K@Z 10001d80 f   flexcan.obj
 0001:00000e24       ?Deinitialize@FlexCAN@@AAAXXZ 10001e24 f   flexcan.obj
 0001:00000f54       ?IST@FlexCAN@@CAKPAX@Z     10001f54 f   flexcan.obj
 0001:000010fc       ?SetupInterruptHandler@FlexCAN@@AAAHXZ 100020fc f   flexcan.obj
 0001:00001200       ?GetBitrate@FlexCAN@@QAAKXZ 10002200 f   flexcan.obj
 0001:00001244       ?SetBitrate@FlexCAN@@QAAKK@Z 10002244 f   flexcan.obj
 0001:00001334       ?AbortTransmission@FlexCAN@@AAAKE@Z 10002334 f   flexcan.obj
 0001:00001448       ?TransmitPacket@FlexCAN@@QAAKPAUCAN_PACKET@@@Z 10002448 f   flexcan.obj
 0001:00001808       ?ReceivePacket@FlexCAN@@QAAKPAUCAN_PACKET@@@Z 10002808 f   flexcan.obj
 0001:00001a0c       ??1FlexCAN@@QAA@XZ         10002a0c f   flexcan.obj
 0001:00001a1c       ?InitFlexCAN@FlexCAN@@AAAXXZ 10002a1c f   flexcan.obj
 0001:00001c30       ?Initialize@FlexCAN@@AAAHPBG@Z 10002c30 f   flexcan.obj
 0001:00001d38       ??0FlexCAN@@QAA@PBG@Z      10002d38 f   flexcan.obj
 0001:00001d88       ??0Settings@@QAA@PBG@Z     10002d88 f   settings.obj
 0001:00001ee8       ??1Settings@@QAA@XZ        10002ee8 f   settings.obj
 0001:00001eec       ?SetupHardware@FlexCAN@@AAAHK@Z 10002eec f   flexcan_pdd:pdd.obj
 0001:00002108       ?LEDBlinker@FlexCAN@@CAKPAX@Z 10003108 f   flexcan_pdd:pdd.obj
 0001:00002170       CeCloseCallerBuffer        10003170 f   coredll:COREDLL.dll
 0001:00002180       CeFreeAsynchronousBuffer   10003180 f   coredll:COREDLL.dll
 0001:00002190       CeAllocDuplicateBuffer     10003190 f   coredll:COREDLL.dll
 0001:000021a0       CeFreeDuplicateBuffer      100031a0 f   coredll:COREDLL.dll
 0001:000021b0       DisableThreadLibraryCalls  100031b0 f   coredll:COREDLL.dll
 0001:000021c0       SetLastError               100031c0 f   coredll:COREDLL.dll
 0001:000021d0       CeAllocAsynchronousBuffer  100031d0 f   coredll:COREDLL.dll
 0001:000021e0       CeOpenCallerBuffer         100031e0 f   coredll:COREDLL.dll
 0001:000021f0       EventModify                100031f0 f   coredll:COREDLL.dll
 0001:00002200       CloseHandle                10003200 f   coredll:COREDLL.dll
 0001:00002210       TerminateThread            10003210 f   coredll:COREDLL.dll
 0001:00002220       WaitForSingleObject        10003220 f   coredll:COREDLL.dll
 0001:00002230       InterruptDisable           10003230 f   coredll:COREDLL.dll
 0001:00002240       KernelIoControl            10003240 f   coredll:COREDLL.dll
 0001:00002250       CreateThread               10003250 f   coredll:COREDLL.dll
 0001:00002260       DeleteCriticalSection      10003260 f   coredll:COREDLL.dll
 0001:00002270       GetLastError               10003270 f   coredll:COREDLL.dll
 0001:00002280       InterruptDone              10003280 f   coredll:COREDLL.dll
 0001:00002290       DevicePowerNotify          10003290 f   coredll:COREDLL.dll
 0001:000022a0       CeSetThreadPriority        100032a0 f   coredll:COREDLL.dll
 0001:000022b0       InterruptInitialize        100032b0 f   coredll:COREDLL.dll
 0001:000022c0       CreateEventW               100032c0 f   coredll:COREDLL.dll
 0001:000022d0       LeaveCriticalSection       100032d0 f   coredll:COREDLL.dll
 0001:000022e0       EnterCriticalSection       100032e0 f   coredll:COREDLL.dll
 0001:000022f0       InitializeCriticalSection  100032f0 f   coredll:COREDLL.dll
 0001:00002300       RegCloseKey                10003300 f   coredll:COREDLL.dll
 0001:00002310       wsprintfW                  10003310 f   coredll:COREDLL.dll
 0001:00002320       RegQueryValueExW           10003320 f   coredll:COREDLL.dll
 0001:00002330       OpenDeviceKey              10003330 f   coredll:COREDLL.dll
 0001:00002340       MmUnmapIoSpace             10003340 f   ceddk:CEDDK.dll
 0001:00002350       MmMapIoSpace               10003350 f   ceddk:CEDDK.dll
 0001:00002360       DDKGpioWriteDataPin        10003360 f   cspddk:CSPDDK.dll
 0001:00002370       DDKGpioSetConfig           10003370 f   cspddk:CSPDDK.dll
 0001:00002380       DDKClockSetGatingMode      10003380 f   cspddk:CSPDDK.dll
 0001:00002390       DDKIomuxSelectInput        10003390 f   cspddk:CSPDDK.dll
 0001:000023a0       DDKIomuxSetPadConfig       100033a0 f   cspddk:CSPDDK.dll
 0001:000023b0       DDKIomuxSetPinMux          100033b0 f   cspddk:CSPDDK.dll
 0001:000024c4       _DllMainCRTStartup         100034c4 f   corelib0:pegdmain.obj
 0001:000024f4       __GSHandlerCheckCommon     100034f4 f   corelib0:gshandler.obj
 0001:00002530       __GSHandlerCheck           10003530 f   corelib0:gshandler.obj
 0001:00002554       __security_init_cookie     10003554 f   corelib0:seccinit.obj
 0001:000025b0       __security_check_cookie    100035b0 f   corelib0:armsecgs.obj
 0001:000025c4       __gsfailure                100035c4 f   corelib0:armsecgs.obj
 0001:00002704       _cexit                     10003704 f   corelib0:cexit.obj
 0001:00002720       _initterm                  10003720 f   corelib0:crt0dat.obj
 0001:00002754       _cinit                     10003754 f   corelib0:crt0dat.obj
 0001:00002788       ??3@YAXPAX@Z               10003788 f   corelib1:COREDLL.dll
 0001:00002798       ??2@YAPAXI@Z               10003798 f   corelib1:COREDLL.dll
 0001:000027a8       memset                     100037a8 f   corelib1:COREDLL.dll
 0001:000027b8       __rt_udiv                  100037b8 f   corelib1:COREDLL.dll
 0001:000027c8       memcpy                     100037c8 f   corelib1:COREDLL.dll
 0001:000027d8       _XcptFilter                100037d8 f   corelib1:COREDLL.dll
 0001:000027e8       __C_specific_handler       100037e8 f   corelib1:COREDLL.dll
 0001:000027f8       __security_gen_cookie2     100037f8 f   corelib1:COREDLL.dll
 0001:00002808       __report_gsfailure         10003808 f   corelib1:COREDLL.dll
 0001:00002818       free                       10003818 f   corelib1:COREDLL.dll
 0001:00002828       InterlockedExchange        10003828 f   coredll:COREDLL.dll
 0001:00002838       TerminateProcess           10003838 f   coredll:COREDLL.dll
 0001:00002860       __IMPORT_DESCRIPTOR_COREDLL 10003860     coredll:COREDLL.dll
 0001:00002874       __IMPORT_DESCRIPTOR_CEDDK  10003874     ceddk:CEDDK.dll
 0001:00002888       __IMPORT_DESCRIPTOR_CSPDDK 10003888     cspddk:CSPDDK.dll
 0001:0000289c       __NULL_IMPORT_DESCRIPTOR   1000389c     coredll:COREDLL.dll
 0002:00000000       __imp_MmUnmapIoSpace       10004000     ceddk:CEDDK.dll
 0002:00000004       __imp_MmMapIoSpace         10004004     ceddk:CEDDK.dll
 0002:00000008       \177CEDDK_NULL_THUNK_DATA  10004008     ceddk:CEDDK.dll
 0002:0000000c       __imp_CeFreeDuplicateBuffer 1000400c     coredll:COREDLL.dll
 0002:00000010       __imp_DisableThreadLibraryCalls 10004010     coredll:COREDLL.dll
 0002:00000014       __imp_SetLastError         10004014     coredll:COREDLL.dll
 0002:00000018       __imp_CeAllocAsynchronousBuffer 10004018     coredll:COREDLL.dll
 0002:0000001c       __imp_CeOpenCallerBuffer   1000401c     coredll:COREDLL.dll
 0002:00000020       __imp_EventModify          10004020     coredll:COREDLL.dll
 0002:00000024       __imp_CloseHandle          10004024     coredll:COREDLL.dll
 0002:00000028       __imp_TerminateThread      10004028     coredll:COREDLL.dll
 0002:0000002c       __imp_WaitForSingleObject  1000402c     coredll:COREDLL.dll
 0002:00000030       __imp_InterruptDisable     10004030     coredll:COREDLL.dll
 0002:00000034       __imp_KernelIoControl      10004034     coredll:COREDLL.dll
 0002:00000038       __imp_CreateThread         10004038     coredll:COREDLL.dll
 0002:0000003c       __imp_DeleteCriticalSection 1000403c     coredll:COREDLL.dll
 0002:00000040       __imp_CeAllocDuplicateBuffer 10004040     coredll:COREDLL.dll
 0002:00000044       __imp_InterruptDone        10004044     coredll:COREDLL.dll
 0002:00000048       __imp_DevicePowerNotify    10004048     coredll:COREDLL.dll
 0002:0000004c       __imp_CeSetThreadPriority  1000404c     coredll:COREDLL.dll
 0002:00000050       __imp_InterruptInitialize  10004050     coredll:COREDLL.dll
 0002:00000054       __imp_CreateEventW         10004054     coredll:COREDLL.dll
 0002:00000058       __imp_LeaveCriticalSection 10004058     coredll:COREDLL.dll
 0002:0000005c       __imp_EnterCriticalSection 1000405c     coredll:COREDLL.dll
 0002:00000060       __imp_InitializeCriticalSection 10004060     coredll:COREDLL.dll
 0002:00000064       __imp_RegCloseKey          10004064     coredll:COREDLL.dll
 0002:00000068       __imp_wsprintfW            10004068     coredll:COREDLL.dll
 0002:0000006c       __imp_RegQueryValueExW     1000406c     coredll:COREDLL.dll
 0002:00000070       __imp_OpenDeviceKey        10004070     coredll:COREDLL.dll
 0002:00000074       __imp_CeFreeAsynchronousBuffer 10004074     coredll:COREDLL.dll
 0002:00000078       __imp_GetLastError         10004078     coredll:COREDLL.dll
 0002:0000007c       __imp_CeCloseCallerBuffer  1000407c     coredll:COREDLL.dll
 0002:00000080       __imp_TerminateProcess     10004080     coredll:COREDLL.dll
 0002:00000084       __imp_InterlockedExchange  10004084     coredll:COREDLL.dll
 0002:00000088       __imp_free                 10004088     corelib1:COREDLL.dll
 0002:0000008c       __imp___report_gsfailure   1000408c     corelib1:COREDLL.dll
 0002:00000090       __imp_??3@YAXPAX@Z         10004090     corelib1:COREDLL.dll
 0002:00000094       __imp_??2@YAPAXI@Z         10004094     corelib1:COREDLL.dll
 0002:00000098       __imp_memset               10004098     corelib1:COREDLL.dll
 0002:0000009c       __imp___rt_udiv            1000409c     corelib1:COREDLL.dll
 0002:000000a0       __imp_memcpy               100040a0     corelib1:COREDLL.dll
 0002:000000a4       __imp__XcptFilter          100040a4     corelib1:COREDLL.dll
 0002:000000a8       __imp___C_specific_handler 100040a8     corelib1:COREDLL.dll
 0002:000000ac       __imp___security_gen_cookie2 100040ac     corelib1:COREDLL.dll
 0002:000000b0       \177COREDLL_NULL_THUNK_DATA 100040b0     coredll:COREDLL.dll
 0002:000000b4       __imp_DDKIomuxSetPadConfig 100040b4     cspddk:CSPDDK.dll
 0002:000000b8       __imp_DDKIomuxSelectInput  100040b8     cspddk:CSPDDK.dll
 0002:000000bc       __imp_DDKClockSetGatingMode 100040bc     cspddk:CSPDDK.dll
 0002:000000c0       __imp_DDKGpioSetConfig     100040c0     cspddk:CSPDDK.dll
 0002:000000c4       __imp_DDKGpioWriteDataPin  100040c4     cspddk:CSPDDK.dll
 0002:000000c8       __imp_DDKIomuxSetPinMux    100040c8     cspddk:CSPDDK.dll
 0002:000000cc       \177CSPDDK_NULL_THUNK_DATA 100040cc     cspddk:CSPDDK.dll
 0002:000000d0       ?dpCurSettings@@3U_DBGPARAM@@A 100040d0     DebugZones.obj
 0002:00000514       __security_cookie          10004514     corelib0:seccinit.obj
 0002:00000518       __security_cookie_complement 10004518     corelib0:seccinit.obj
 0002:00000520       _exitflag                  10004520     corelib0:cexit.obj
 0002:00000524       __onexitend                10004524     <common>
 0002:00000528       __onexitbegin              10004528     <common>
 0002:0000052c       g_pcsExit                  1000452c     <common>
 0002:00000530       _pRawDllMain               10004530     <common>

 entry point at        0001:000024c4

 Static symbols

 0001:000023c8       _DllMainCRTStartupHelper   100033c8 f   corelib0:pegdmain.obj
 0001:00002608       doexit                     10003608 f   corelib0:cexit.obj
